:060000000200860225E764
:03000B00021EE2F0
:03001300021DC902
:03001B00021FDCE5
:0300230002258C27
:10002B00324C6967687443756520534D50544520B5
:10003B00496E7465726661636520202863292031DF
:10004B003939352020416C636F726E204D634272DB
:10005B0069646520496E632E0D4C6967687443753E
:10006B006520534D50544520496E7465726661632B
:10007B006520012056322E30300D00C2AF75D000F6
:10008B0075816943B0FF4390FF75892175880475AD
:10009B008DFF758BFFD28E7589237598D0787FE491
:1000AB00F6D8FD751800751E149000007400F0A3AF
:1000BB00A883B81FF9D2B4D29612010090278E12E2
:1000CB0001B49027A11201B412180F75B80075A8CE
:1000DB0011D2AF751296C201758169758300758255
:1000EB0000C083C082120251D082D083D583F2D557
:1000FB0082EF02134390000075A0A07802E230E774
:10010B000BA3E583B405F6C238020151D2387A301D
:10011B001201527A301201527A381201527A80123D
:10012B0001527A061201527A0C1201527A01120113
:10013B00527A401201527A5A1201717A40120152CC
:10014B00120193B45AC122C0F030381775F0007504
:10015B00A0A07802E230E70700D5F0F302016E7839
:10016B0000EAF2D0F022C0F030381A75F00075A01A
:10017B00A07802E230E70700D5F0F302019075A0FA
:10018B00A07801EAF2D0F022C0F030381975F000F7
:10019B0075A0A07802E230E70700D5F0F30201B1B9
:1001AB0075A0A07803E2D0F022740093A31201D2C1
:1001BB00FA740093A32AFA120152740093A36006F7
:1001CB00FA12017180F42283227FBF93D37A8512B6
:1001DB000152E55175F000600475F00A842430FA81
:1001EB00120171E5F02430FA1201717A3A120171A1
:1001FB00E55275F000600475F00A842430FA1201A0
:10020B0071E5F02430FA1201717A3A120171E5535B
:10021B0075F000600475F00A842430FA120171E560
:10022B00F02430FA1201717A2E120171E55475F037
:10023B0000600475F00A842430FA120171E5F02491
:10024B0030FA12017122E559655A70030203777572
:10025B00A016A959E37004055980EB75A017E35458
:10026B003F23239002727302037200020378000291
:10027B000372000203720002037200020372000297
:10028B000372000203720002037200020372000287
:10029B000372000203720002037200020372000277
:1002AB000372000203720002037200020372000267
:1002BB000372000203720002037200020372000257
:1002CB000372000203720002037200020372000247
:1002DB000372000203720002037200020372000237
:1002EB000372000203720002037200020372000227
:1002FB000372000203720002037200020372000217
:10030B000372000203720002037200020372000206
:10031B0003720002037200020372000203720002F6
:10032B0003720002037200020372000203720002E6
:10033B0003720002037200020372000203720002D6
:10034B0003720002037200020372000203720002C6
:10035B0003720002037200020372000203720002B6
:10036B000372000203720005590202512230383B1E
:10037B008559820582E582655A6032758316E07075
:10038B002A758317E070EC8559820582E00582128D
:10039B0001D2FAE005822AFA120152E005826006C8
:1003AB00FA12017180F58582598002055902037793
:1003BB00E559655A60081203EB20232380F2302D98
:1003CB00051222C4800BE5636564600512050C8081
:1003DB00F5E55F6560600812052C80F585605F228E
:1003EB0075A017A959E3FA75A016E3FB0559C229A5
:1003FB00BB0006EA20280F803CEA30E73690155800
:10040B00F0D22802050BC228B4FE0DF51CF51D75A4
:10041B001800751E1402050BB480005005751D00E5
:10042B00805E751DFDD224901559C0E0E4F0D0E03C
:10043B000204C8D229AD1DBDFE03020457BD000343
:10044B000204A7BDFD030204C802050BBB0002801A
:10045B001AF5F0901558E0251CC313B5F005D223FF
:10046B0002050B745512131802050B851EA0A81854
:10047B00F2251CF51C088818B80002051E02050B96
:10048B00901558E075831E856282F0740175831E8A
:10049B00F00582E5616582602185826275831E8528
:1004AB006282EAF0EB75831EF00582E5616582607E
:1004BB00098582629060057406F002050B302909EC
:1004CB00901559E0C313FAC229901559E02AF0751B
:1004DB00831C855E82EAF0302406C22474018002FC
:1004EB00740075831BF00582E55D6582600F858264
:1004FB005E90800274B5F09080057406F002050BD7
:10050B002275A01DA863E20563758319855C82F0D3
:10051B000582E55B6582600385825C202002D299AF
:10052B002275A01AA85FE2055FB4FE0BD230C23170
:10053B00C232C2330205D830300AB41302D231C2F0
:10054B00300205D8303110B42000505C90155FF0AC
:10055B00C231D2320205D830320A901560F0C23265
:10056B00D2338069303349F87A1190155FE02AFA5B
:10057B00901560E02A547FC398702D901560E0F8B9
:10058B0090155FE09015612582F58274003583F537
:10059B0083E8F030E504D234800375671E90151E96
:1005AB00E054FDF090E000F0C231C232C233801D46
:1005BB00C231C232C233758319855C82F00582E584
:1005CB005B6582600385825C202002D2992290E8D1
:1005DB0000E0F890E000E058C0E075A015781AE252
:1005EB00FAD0E0F26A5AFAEA540F604830E018D2B7
:1005FB0091C200C201A215C2154039302213301F1F
:10060B001012168C02063F30E107202B04D200C2D9
:10061B009130E304D201801C30221130E402D21558
:10062B0030E211D201D291121A83800830E205D246
:10063B0001121A83227851E60846084608466012D2
:10064B0012065E7002800B1206ED60067D16DDFE53
:10065B0080F522900000E06026F975650030257D5D
:10066B0020267A7E107F008E828F83E0B4FF02807B
:10067B006CF5F07851E6B5F00280104060D902803D
:10068B005C74082EFEEF3400FF80DCA3E0B4FF02A5
:10069B00804BF5F008E6B5F0028004404080DEA305
:1006AB00E0B4FF028037F5F008E6B5F002800440B5
:1006BB002C80CAA3E0B4FF028023F5F008E6B5F066
:1006CB00028004401880B6E565B4000DA3AB82AC84
:1006DB008390151CEBF0A3ECF0056580A0C227E519
:1006EB00652290151CE0FBA3E0FCE565B40003025A
:1006FB0007378B828C83E0FEA3E0FFA3E0F9700346
:10070B00020726A3E0B4FF0302073AB480005003AC
:10071B0002076A0207C8D565028011EB2408FB901B
:10072B00151CF0A3EC3400FCF00206FDE56522E598
:10073B005CC3955BF489F0B5F00050030207378E6C
:10074B00828F83A85C75A019E0F2058208D9F9881D
:10075B005C202002D299D56503020737020726E5F4
:10076B0062C39561F489F0B5F00050030207378E30
:10077B00828F83A86275A01EE0D2E7F275A01E746B
:10078B0001F2D903088025058208D9028010E07593
:10079B00A01EF275A01E7400F2058208D9F0E07558
:1007AB00A01EF275A01E7401F2058208886290608B
:1007BB00057406F0D56503020737020726E55EC30D
:1007CB00955DF489F0B5F00050030207378E828FE8
:1007DB0083A85EE075A01CF275A01B7401F2058264
:1007EB0008D903020726E075A01CF275A01B740044
:1007FB00F2058208D9F0885E90800274B5F0908083
:10080B00057406F0D56503020737020726E538C4E1
:10081B00540FF5F0E53954F045F030E72530E6227A
:10082B00543FF5F0B43F028024900007E0B5F0028E
:10083B00801B901500E0600AFAA3E0B5F002800D72
:10084B00DAF790153AE4F0A3F0A3F0800890153294
:10085B00E5F0F0D21622901532E0F5F0A3E53AC49C
:10086B00540FF9E53B543049F025F0F5F0A3E53C86
:10087B00C4540FF9E53D543049F025F0543FF5F0E1
:10088B00901532E5F0F022901532E0F5F0E53EC41C
:10089B00540FF9E53F543049B5F002800B90153AEF
:1008AB00E4F0A3F0A3F08020C21E7903783A75A080
:1008BB0015E2F5F0E0B5F0028002D21EF212192C0F
:1008CB00D9EF301E03021934227400B5520DB55303
:1008DB000AB551077403B55400500122901522E05C
:1008EB0060F9FA7400F0A3A85E121BFAB40300407F
:1008FB00F875A01CE0D2E7F2FB75A01B7401F2089F
:10090B0075A01C7408F22BFB75A01B7400F2087504
:10091B00A01CEBF275A01B7400F208885E75A0801A
:10092B00790274B5F375A08079057406F3A3DAB96F
:10093B00C21B22900000E07005D22602099775F0C9
:10094B0000900005E0C395F0900003F075F008905F
:10095B000006E095F0900004F0900000E0C226C382
:10096B0094025002802604FA750513750400850461
:10097B00068505077907120A09EAFB12099A790716
:10098B00120A09DBF67905120A09DAE2D22522C02E
:10099B0082C083A8058504A0850782850683E0F5C0
:1009AB00F0E2C395F0C0D01209E1E0F5F0E2D0D04F
:1009BB0095F0C0D01209E1E0F5F0E2D0D095F0C08F
:1009CB00D01209E1E0F5F0E2D0D095F04003120926
:1009DB00F5D083D08222C0E01582E582B4FF0215E8
:1009EB008318B8FF0215A0D0E0227908E2F5F0E0F9
:1009FB00F2E5F0F0A308B8000205A0D9EF22E72436
:100A0B0008F719E73400F722901400E0B442030210
:100A1B000C5B543F2323900A2573020B2D00020D10
:100A2B005200020DF300020E0400020E2100020B15
:100A3B002500020E3200020E5800020E9200020E2A
:100A4B00B400020FE2000210060002102C0002108C
:100A5B0046000210500002105A000210B900021199
:100A6B00920002116E000211480002111F00020BCE
:100A7B002500020B2500020B2500020B2500020BA3
:100A8B002500020B2500020B2500020B2500020B93
:100A9B002500020B2500020B2500020B2500020B83
:100AAB002500020B2500020B2500020B2500020B73
:100ABB002500020B2500020B2500020B2500020B63
:100ACB002500020B2500020B2500020B2500020B53
:100ADB002500020B2500020B2500020B2500020B43
:100AEB002500020B2500020B2500020B2500020B33
:100AFB002500020B2500020B2500020B2500020B23
:100B0B002500020B2500020B2500020B2500020B12
:100B1B002500020B2500020B25007455121318C279
:100B2B002322901401E0B4FE03020B51B4FF030225
:100B3B000B7FB40003020B7FB4FD03020B7F7455D4
:100B4B00121318C22322120B5C74AA121318C2239D
:100B5B00227A079000007400F0A3DAFCD226D2258B
:100B6B00751800751E14751F007400900005F07445
:100B7B0008A3F022C21EF5F0202606900000E070BC
:100B8B0003020C4AFBF51F7A01A9F0EA75F008A4E1
:100B9B00240FF582E5F03400F58389F0E0B5F0021F
:100BAB008003020C3DD21EE582C39403F582E583DC
:100BBB009400F583E0FCA3E0FDA3E0F9E51FC39AE5
:100BCB0004C0F075F008A4AFF0FEEA1475F008A4A9
:100BDB002410F8E5F03400F5A0EA75F008A4241011
:100BEB00F582E5F03400F583120C87ECF8EDF5A0F7
:100BFB00E92CF58274003DF5837400C39582FE7475
:100C0B00149583FF120C87900003E0C399F0A3E0C7
:100C1B009400F0A3E0C399F0A3E09400F0120C96BB
:100C2B00D0F01B151FE51FB40003020B51BB000CCA
:100C3B00800D0ABB00028007DB028003020B94309D
:100C4B001E06E51F900000F074AA121318C223228F
:100C5B00A85C9000647900E9936017B401037441B8
:100C6B000475A019F20908E8B55BEC2020FAD299BB
:100C7B0080F6885C202002D299C22322E0F212195E
:100C8B002CDEF9BF00028002DFF222900014E51F78
:100C9B006029F8E0C39CAE82AF83A3E09505400DBD
:100CAB008E828F83E0C399F0A3E09400F074072544
:100CBB0082F58274003583F583D8D822900000E04A
:100CCB00F5F0FA7B007E0D900003E02AFA74003BEE
:100CDB00FBA3DEF6900010AEF0BE0003020CF87F13
:100CEB0008E02AFA74003BFBA3DFF6DEF290000368
:100CFB00E0FFA3E0FE900800BF0005BE00028011DC
:100D0B00E02AFA74003BFBA3DFF6BE00028002DE92
:100D1B00EF7E0F901500E02AFA74003BFBA3DEF682
:100D2B007E0B90150FE02AFA74003BFBA3DEF67ED8
:100D3B0020901542E02AFA74003BFBA3DEF69000EC
:100D4B0001EAF0A3EBF022900000E004B4FE08747B
:100D5B0055121318020DF0F014F5F07408A42410BA
:100D6B00F8E5F03400F5A07A04901401E0F21219C2
:100D7B002CDAF9E0B4FE0E900000E014F07455127A
:100D8B001318020DF0FDA3E0FCA3A982AA83900027
:100D9B0003E02CF0A3E03400F0900005E0F5F0F256
:100DAB0012192CE0F2FB12192CECF212192CEDF2A9
:100DBB0012192C74FFF212192CF212192CF21219AF
:100DCB002CF28A838982A9F0E08BA0F3A309B900E6
:100DDB00010BDCF4900005E9F0A3EBF0C226C22571
:100DEB0074AA121318C223222026062025031209E7
:100DFB003E74AA121318C223221218A174AA12133A
:100E0B0018C22320340B90151EE04402F090E00032
:100E1B00F0D297D2962212180F121C5412123D7454
:100E2B00AA121318C22322901401E0B4400040020E
:100E3B008013B40A00400E900007F01218A174AA98
:100E4B0012131880057455121318C2232290140123
:100E5B00E0B40A0040028022FA780075A015F21265
:100E6B00192CE0B43F005012B43200400DF2DAEF0F
:100E7B0074AA1213181218A1800A901500E4F074CA
:100E8B0055121318C22322780175A0149015427DB8
:100E9B0020E2F012192CDDF91218A1121C541212B7
:100EAB003D74AA121318C22322901401E070057529
:100EBB00F0188050B4010575F0198048B40205751F
:100ECB00F01E8040B4030575F01E8038B404057520
:100EDB00F01E80307402900009F090150F7400F032
:100EEB00A37400F0A37400F0A37400F0A37418F0C3
:100EFB00A37400F0A37400F0A37400F074551213E4
:100F0B0018020FD3900009F075A015780F901402FA
:100F1B007955E0B4180050BCF2F7A30809E0B43CD3
:100F2B000050B1F2F7A30809E0B43C0050A6F2F769
:100F3B00A30809E0B5F000509BF2F7A3087930C283
:100F4B0023E0B41804D22380054003020EDFF2F72E
:100F5B00A30809E0B43C004003020EDF3023056018
:100F6B0003020EDFF2F7A30809E0B43C00400302D2
:100F7B000EDF3023056003020EDFF2F7A30809E052
:100F8B00B5F0004003020EDF3023056003020EDFD5
:100F9B00F2F7A3E0A2E09222A2E19205A2E2921F55
:100FAB00A2E3922AA2E4922BA2E5922DA2E6922E24
:100FBB00A2E79213900008F0D296202204C201807F
:100FCB0002D20174AA1213181218A1121C54121275
:100FDB003D121C01C22322901401E0FBA3E0FA9006
:100FEB00151EE04AF0FAA3E04BF090E800F090E019
:100FFB0000EAF074AA121318C22322901401E0F431
:10100B00FBA3E0F4FA90151EE05AF0FAA3E05BF0B4
:10101B0090E800F090E000EAF074AA121318C223D3
:10102B002290E800E0FB90E000E0FA74AA1213189B
:10103B00EB121318EA121318C22322D20174AA124C
:10104B001318C22322C20174AA121318C2232290AE
:10105B001401E0A2E0921D900008E092E3C21D5043
:10106B0002D21DF075A0157817901402E0F9F20862
:10107B00A3E0FAF208A3E0F2FBC3740099748D9A13
:10108B0074279B40030210AEC21D900008E054F77A
:10109B00F09015177400F0A3F0A3F0745512131809
:1010AB000210B61218A174AA121318C223229000B0
:1010BB0000E0FFFA1213189000100FDF02804EE0D1
:1010CB001213182AFAA3E01213182AFAA3E0121328
:1010DB00182AFAA3E01213182AFAA3E0FDA3E0FEE4
:1010EB00A3E0FCA3E0A31213182AFAEC1213182A9C
:1010FB00FAC082C0838D828E830CDC028009E012E1
:10110B0013182AFAA380F3D083D08280AEEA12138D
:10111B0018C223227F037E007A00903400E0121362
:10112B00182AFAA3DEF7DFF59020007E10E01213E9
:10113B00182AFAA3DEF7EA121318C22322901561BC
:10114B007F20E4F0A3DFFC756700C234C235C236E2
:10115B0090151EE04402F090E000F074AA121318F0
:10116B00C22322E430350244013036024402FA1223
:10117B0013189015617F20E01213182AFAA3DFF7DA
:10118B00EA121318C22322901401E0541F75F010B9
:10119B00A42400F582E5F03435F58375A0147801AD
:1011AB001217FAA85E121BFAB4100040F890140143
:1011BB001211EE74AA121318C223227C20EC1475A0
:1011CB00F010A42400F582E5F03435F583E030E728
:1011DB000FA85E121BFAB41000500280F61211EE2B
:1011EB00DCDB22E0D2E775A01CF2FB75A01B7401BF
:1011FB00F20875A01C7400F275A01BF208A37A0DFF
:10120B00E075A01CF22BFB75A01B7400F208A3DA8F
:10121B00EF75A01CEBC313F275A01B7400F20888CA
:10122B005E75A080790274B5F375A080790574069C
:10123B00F322121BFAB4080040F874BF855E827566
:10124B00831CF0FB75831B7401F07403058275839B
:10125B001CF02BFB75831BE4F0058275831CF0756A
:10126B00831BF0058275831CF075831BF0C0829085
:10127B000009E0D082058275831CF02BFB75831B64
:10128B00E4F0E535058275831CF02BFB75831BE4BD
:10129B00F0E534058275831CF02BFB75831BE4F0A2
:1012AB00058275831CEBC313F075831BE4F0058279
:1012BB0085825E90800274B5F09080057406F022F2
:1012CB00FBE55EC3955DF4B4030050030212CCEB57
:1012DB00A85E75A01CF275A01B7401F20875A01C0A
:1012EB00E5F0F22BFB75A01B7400F20875A01CEB4C
:1012FB00C313F275A01B7400F208885E75A0807989
:10130B000274B5F375A08079057406F322C0E0C0B2
:10131B0082C083758319855C82F0E55C04F583B527
:10132B005B072020FAD29980F685835C202002D2BD
:10133B0099D083D082D0E02275A890C28CC28EC285
:10134B008F9027B41201B49027C41201B49027ECEC
:10135B001201B4C20BC20DC212C20FC20CC210C218
:10136B000EC207851211758A00754C0075294075E0
:10137B002A01755500755600755700755800753361
:10138B0000901517E0F530A3E0F531A3E0F532C27C
:10139B00AF75B80675A81ED246D28CD2AFC2231237
:1013AB000251100C0280F8E539540375F00AA4F8C9
:1013BB00E538540F28200E09B415E4D20E7A0080BC
:1013CB00DEF89013D5EA540323738006800A800E4F
:1013DB008030B8162B0A80C7B817250A80C1B818F9
:1013EB00030A80BBB8001975461875127875295B0E
:1013FB00C20690282F1201B47400900009F080628D
:10140B00805BB8193C75461E751296752915C20678
:10141B009028411201B47402900009F0E53930E2D2
:10142B0010D20690284A1201B47404900009F0807F
:10143B0031C2069028531201B47404900009F08055
:10144B0021B8001975461975127D75294DC2069084
:10145B0028381201B47401900009F08005C20E0205
:10146B0013AA9027D21201B4C2AF854341854442DF
:10147B00D2AFE54175F014A4F541A8F0E54275F043
:10148B0014A428F542754E00754D00D210D20FE50D
:10149B0039540375F00AA4F5F0E538540F25F00420
:1014AB00F548F554E53B540775F00AA4F5F0E53A19
:1014BB00540F25F0F549F553E53D540775F00AA493
:1014CB00F5F0E53C540F25F0F54AF552E53F540392
:1014DB0075F00AA4F5F0E53E540F25F0F54BF551E8
:1014EB00C202C218C219740A120251301902C2196F
:1014FB00301823C218300D089027D21201B4801671
:10150B009027DF1201B4D296121D08D51108D236DE
:10151B00C201C2228012300208C202121D0812013F
:10152B00D83017C4C21780C01217E7D2970200E356
:10153B0075A891C28CC28EC215C21AC21890151E04
:10154B00E054FEF090E000F012168C20423920415E
:10155B001B20400C90155075461875400002159FC6
:10156B0090155275461975400002159F30400C902E
:10157B00155675461E75400002159F9015547546FD
:10158B001E75400C02159F90155475461E7540082C
:10159B00C240C241E0A3750F00F50EE0F50D754793
:1015AB0000750936750C00750B0A750A01D2098591
:1015BB000E4F1217E7C2AF75B802850E8A202E07A1
:1015CB0075A81BD28C800575A81FC28BC246C28D15
:1015DB00C28FD2AFC223740AF5661203BB30230647
:1015EB00120A1320012230020BC2021206403013E2
:1015FB0003121D083018E3C2181205D92001093057
:10160B001504C292800E80D275A891C28CC28E75C1
:10161B002800805D1203BB20233430022AC2021241
:10162B0005D920013E20151FD2927536FC7537BFA8
:10163B00750936750C00750B0A750A01D209D20BA8
:10164B00C20AC2070215563018CAC21880C6D291F8
:10165B0075A891C28CC28EC215D201752800120AD0
:10166B0013800ED29175A891C28CC28EC2157528AB
:10167B000090151EE04401F090E000F0D2960200BD
:10168B00E31217E790150FE0F555F54BA3E0F55670
:10169B00F54AA3E0F557F549A3E0F558F54800A343
:1016AB00E0F530A3E0F531A3E0F532A3E0F533909C
:1016BB000009E070087528007568048027B40108DC
:1016CB00752801756804801CB403087528047568B7
:1016DB00018011B40408752802756801800675280D
:1016EB00037568017536FC7537BFE54875F00A84DC
:1016FB0085F0384540F539E54975F00A8485F03AAF
:10170B00F53BE54A75F00A8485F03CF53DE54B75F4
:10171B00F00A8485F03EF53F2290400374C2C2AFBD
:10172B00F0904000E0E0F4FCE0F4FD9040037436F0
:10173B00F0904000E4F0F0D2AF202C43ED13547F37
:10174B00FDEC132403FCED3400FDC3E5349CFC904D
:10175B006003F0E5359DFD906003F075F00030E718
:10176B000375F0FFAEF0C390155AE03CFCF0A3E01C
:10177B003DFDF0A3E03EFEF020E70C4D4C702EC279
:10178B002CAD2CAC2D804775F00AF47013EDF47072
:10179B000FECF4B45000500803030303540FF5F09F
:1017AB00E52CC395F0FDE52D9400FC802175F00A26
:1017BB00EE7011ED700EECB45000500803030303F0
:1017CB00540FF5F0E52C25F0FDE52D3400FC75A04C
:1017DB00407801EDC2AFF2ECF2D2AF22D22CE49002
:1017EB00155AF0A3F0A3F0AD2CAC2D1217D9227A19
:1017FB0010800312192CE2F0DAF9FAE0C39A70FBAD
:10180B0012192C22120B5C121858D2357D04785504
:10181B0090150FE0F6A308DDFA7D047830901513D0
:10182B00E0F6A308DDFA900008E0A2E09222A2E124
:10183B009205A2E2921FA2E3922AA2E4922BA2E5C6
:10184B00922DA2E6922EA2E79213C201229027526A
:10185B0075A00078007A10E493F212192CDAF89044
:10186B00276275A01578007A0FE493F212192CDA1F
:10187B00F890278375A015780F7A0BE493F2121961
:10188B002CDAF890276D75A01578427A16E493F24E
:10189B0012192CDAF82220260620250312093E12F3
:1018AB000CC7780075A000902000E2FC1217FAEC30
:1018BB0070030218F5C31304FC1217FADCFB90003B
:1018CB0003E0FCFFA3E0FD7A04EDC313FDEC13FC76
:1018DB00DAF7EF540F60010CBC0002800D78007535
:1018EB00A0089028001217FADCFB780075A0159061
:1018FB0034001217FA780F75A0159034101217FADE
:10190B00784275A0159034201217FA785275A015ED
:10191B009034301217FA9034407455F0E0B455FC03
:10192B0022A308B8000205A022901533E0540F2320
:10193B0023901940730219810002199B00021A8728
:10194B0000021ADC00021B0100021B0D00021B1916
:10195B0000021B2500021B9000021BAA00021BC4E5
:10196B0000021BDF0002198000021980000219809F
:10197B00000219800022901533E05430FA334A5498
:10198B0050FAA3E0543F901520F0901521EAF02275
:10199B00901534E0543FD2E7FA901520E0F99015FA
:1019AB0021E0F5F0301D048A588933121BFAB40577
:1019BB000040F875831C855E82EAF075831B740109
:1019CB00F0058275831C7401F02AFA75831B740071
:1019DB00F0058275831CE5F0644003542045F0202C
:1019EB002207200D09440880053001024408F02A23
:1019FB00FA75831B7400F0058275831CE9543FF064
:101A0B002AFA75831B7400F0058275831CEA035454
:101A1B007FF075831B7401F0058285825E908002D6
:101A2B0074B5F09080057406F0C22122121BFAB433
:101A3B000300500280F675831C855E82EAF0758385
:101A4B001B7401F0058275831C7408F02AFA7583E8
:101A5B001B7400F0058275831CEA03547FF07583B9
:101A6B001B7401F0058285825E90800274B5F09044
:101A7B0080057406F0C22122743F8006C2219015A6
:101A8B0034E0543FD2E7FA121BFAB4030050028041
:101A9B00F675831C855E82EAF075831B7401F00575
:101AAB008275831C7408F02AFA75831B7400F00589
:101ABB008275831CEA03547FF075831B7401F00558
:101ACB008285825E90800274B5F09080057406F07A
:101ADB0022901534E0543FFA901522E0B40A0280AC
:101AEB001204F0F9E58229F58274003583F583EA57
:101AFB00F0D21BC22122901534E0543FFA79180220
:101B0B001B31901534E0543FFA7919021B319015B3
:101B1B0034E0543FFA791A021B31901534E0543FEC
:101B2B00FA791B021B31E562C39561F4B4050050D1
:101B3B000280F375831E75A01E85628274FF44803C
:101B4B00FBF07401A882F205827400F02BFB740089
:101B5B00A882F20582E9547FF02BFB7400A882F275
:101B6B000582EAF02BFB7400A882F20582EB03548A
:101B7B007FF07401A882F205828582629060057401
:101B8B0006F0C22122901533E0232354C0F9A3E0C1
:101B9B00543F49F990151EE049F090E000F0229077
:101BAB001533E0232354C0F9A3E0543F49F99015B2
:101BBB001FE049F090E800F022901533E023235406
:101BCB00C0F9A3E0543F49F4F990151EE059F09089
:101BDB00E000F022901533E0232354C0F9A3E05426
:101BEB003F49F4F990151FE059F090E800F022E519
:101BFB005EC3955DF4229060027415F09060002036
:101C0B002D04741B80027413F07407F0A3202D04B1
:101C1B0074BB800274CCF09060047408F090600286
:101C2B007405F09060057406F09080027415F090C6
:101C3B008000741BF07407F0A374CCF090800474D4
:101C4B0008F09080057404F0221217E7C203901578
:101C5B0042E0F52B6002D203A3A3A3E0F52DA3E092
:101C6B00C0E054FEC39432F52CE52D9400F52D9075
:101C7B0040037476F09040017F32E52C2402F52C62
:101C8B00F0E52D3400F52DF0122749DFED7F19E536
:101C9B002CC39402F52CF0E52D9400F52DF01227B2
:101CAB0049DFECD0E0F52CF0E52DF074E775F00092
:101CBB007F081226F0903421E0F5F0A3E07F10129C
:101CCB0026F0A3E0F5F0A3E07F0F1226F0D297A346
:101CDB00F52D121CE122900009E0B4000590154887
:101CEB008013B4010590154A800BB4020590154E74
:101CFB00800390154CE0F535A3E0F53422C0D0C03D
:101D0B00E0C0F0C082C083E55CC3955BF4B4070010
:101D1B005003021DBE758319855C8274BFF0F5F00C
:101D2B007583187401F00582758319740DF025F015
:101D3B00F5F0758318E4F00582758319E54BF025F2
:101D4B00F0F5F0758318E4F00582758319E54AF018
:101D5B0025F0F5F0758318E4F00582758319E549D4
:101D6B00F025F0F5F0758318E4F00582758319E51D
:101D7B0048F025F0F5F0758318E4F00582C08290E9
:101D8B000009E0D082547F300D024480758319F036
:101D9B0025F0F5F0758318E4F00582758319E5F0ED
:101DAB0003547FF0758318E4F0058285825C202054
:101DBB0002D299D083D082D0F0D0E0D0D02220466E
:101DCB0003D28C32C0D0C0E0D2147402C28CC58A4C
:101DDB00D28CF54FE4C54C308D070470027403C2EE
:101DEB008DF550C3E54F948AE5509400401BC3E535
:101DFB0029954FE52A95504004D208801374B59568
:101E0B004F74029550C2085007C20BC20D021EDD63
:101E1B0030080D30070A200A28C2070547021EDDCD
:101E2B00200B69A208E53713F537E53613F536B401
:101E3B00FC76E537B4BF71300807D20AD207021E11
:101E4B00DDC2B4D2177400B54808B54905B54A02CE
:101E5B008014E53F540775F00AA4F5F0E53E540FE6
:101E6B0025F0F54BF551750938750B08750A087592
:101E7B004700D20BC20AC207300F57754500754E8B
:101E8B0000754D00D28ED28FC20F8046C000A208C3
:101E9B00A809E613F6D000D50A0E0509750A08D570
:101EAB000B06C20BD20DD20C300804D207802305CF
:101EBB0047C207E54354F02544C4F50FE54F54F0F2
:101ECB002550C4254350020544C3950FF5435002DA
:101EDB001544D0E0D0D032204603021EF8C0E005F6
:101EEB004CE54C7005D204754C03D0E032C0D0C029
:101EFB00E0C0F0C082C083300911301507300504F3
:101F0B00D2968002B296C207021FA7C000A809E6AC
:101F1B0030E00E301507300504D2968002B296D20F
:101F2B000703F6D0000547E50AC333F50A506D7574
:101F3B000A010509D50B65750936750B0A7547003E
:101F4B00854854854953854A52854B51E54875F070
:101F5B000A8485F0384540F539E54975F00A8485E2
:101F6B00F03AF53BE54A75F00A8485F03CF53DE522
:101F7B004B75F00A8485F03EF53FD28F302E1DD580
:101F8B00681AB209050CC28C758AFE756801E528C2
:101F9B005407B40200502F756804802AB209850ECD
:101FAB004FE50CC3950D4002054F050CC28CE4C3E5
:101FBB00954F258AF58AD28C201A0BE509B43B067E
:101FCB00D21AD218D2B4D083D082D0F0D0E0D0D0F5
:101FDB0032204603022231C0D0C0E0E54E6004152A
:101FEB004E8019E54D601AC3E4954D754D00C28EB8
:101FFB00258C5004D28E8009F58CD28ED0E0D0D0B7
:10200B0032C21AE5457007200D0DC2B48009B40227
:10201B0006D21AD2B4D218C0F0C083C082200D03EE
:10202B00022166201A0C101406C20DC20BD20F022D
:10203B00216653A8FB854C17858A16E547A20785B1
:10204B00441485431543A8049211F5F0B4280302F8
:10205B00206250030220E5942823F5139415400BBE
:10206B00C20DC212C20BD20F022166E514C313C5F7
:10207B001513F51420110BC39516E5159517400292
:10208B0080020513E5148513F0A4F51685F017E50A
:10209B00158513F0A42517C313C51613C516C31343
:1020AB00F517E51613F516E517C313F515E5161316
:1020BB00C515C313C51513F514C3E5419514F541A7
:1020CB00E5429515F542C3E5419516F54DE542956B
:1020DB0017F54E154ED21202216EC3742895F023BC
:1020EB00F5139415400BC20DC212C20BD20F022175
:1020FB0066E514C313C51513F51420110BC3951600
:10210B00E5159517400280021513E5148513F0A40D
:10211B00F51685F017E5158513F0A42517C313C520
:10212B001613C516C313F517E51613F516E517C3E6
:10213B0013F515E51613C515C313C51513F514259E
:10214B0041F541E5153542F542E5162541F54DE5DD
:10215B00173542F54E154ED212800885424E8541F9
:10216B004D154EE545B403028008B40102D21902A5
:10217B002221300D4F30124CC297851211E5395484
:10218B000375F00AA4F5F0E538540F25F0F548E592
:10219B003B540775F00AA4F5F0E53A540F25F0F51A
:1021AB0049E53D540775F00AA4F5F0E53C540F25BD
:1021BB00F0F54A7400B54811B5490EB54A0B054800
:1021CB00054B8040D2971217E70548E548B54634D2
:1021DB007548000549E549B43C2A754900054A3064
:1021EB000610E54A75F00A84E5F06006740225488E
:1021FB00F548E54AB43C0D754A00054BE54BB41860
:10220B0003754B00E548F554E549F553E54AF5529E
:10221B00E54BF551D2020545534503D082D083D00F
:10222B00F0D0E0D0D032C0D0C0E0C0F03015030207
:10223B0022A40548E548B546347548000549E549EB
:10224B00B43C2A754900054A30411020400DE54A3F
:10225B0075F00A84C5F06003754802E54AB43C0D7D
:10226B00754A00054BE54BB41803754B00E54BB5B0
:10227B003027E54AB53122E549B5321DE548B5337E
:10228B0018302B02D201300004D201D29185554B6C
:10229B0085564A855749855848D202C21AC2B4C0DE
:1022AB0083C08290151EE04401F090E000F0D082D4
:1022BB00D083D0F0D0E0D0D032E564C39563856392
:1022CB001BB407005003022581122582B4F066125D
:1022DB00258220E75EB47F5D12258220E755B47F0F
:1022EB0002800B2409F5F0900007E0B5F0471225AA
:1022FB008220E73FB4023E12258220E736B410025B
:10230B008008B430028003B47F2B12258220E72390
:10231B00F51AB401028021B40202801CB4030280BE
:10232B0017B415030223BFB416030223BFB417055A
:10233B000223BF151B02257BE564C39563B40F0015
:10234B00500302258112258220E7E8C3943075F0F3
:10235B000AA4F51C12258220E7D9C39430251CF55D
:10236B001C12258220E7CCB400CB12258220E7C3B8
:10237B00C39430F51D12258220E7B8B400B712259F
:10238B008220E7AFC3943075F00AA4F51E122582A4
:10239B0020E7A0C39430251E75F00AA4F51E85F026
:1023AB001F12258220E78CC39430251EF51EE51FD6
:1023BB003400F51F12258230E721B4F721E51AB45A
:1023CB000104C2018033B40302802EB40203022441
:1023DB00A0B4150DC201C2150224F102257B022304
:1023EB003EB4160AD2013022EFD2150224F1B417F3
:1023FB0005D2010224F102257B121BFAB405005011
:10240B000280F675831C855E82E51C4480F519B449
:10241B0081004000F075831B7401F0058275831CED
:10242B007401F02519F51975831B7400F00582757D
:10243B00831CE51E33E51F3330E20244105413C5F1
:10244B001D600920E104744080027420451DF51DB8
:10245B00E51AB403067408451DF51DE51DF0251995
:10246B00F51975831B7400F0058275831CE51E54EA
:10247B007FF02519F51975831B7400F005827583A0
:10248B001CE51903547FF075831B7401F0058285DD
:10249B00825E0224E5121BFAB40300500280F6752B
:1024AB00831C855E82E51C4480F519F075831B74D3
:1024BB0001F0058275831C7408F02519F5197583D5
:1024CB001B7400F0058275831CE51903547FF075AE
:1024DB00831B7401F0058285825E90800274B5F0D7
:1024EB009080057406F074F075831E856282F0741B
:1024FB000075831EF00582E56165826073858262DB
:10250B00747F75831E856282F0740075831EF005DF
:10251B0082E56165826059858262740375831E85CD
:10252B006282F0740075831EF00582E5616582603E
:10253B003F858262740275831E856282F07400751A
:10254B00831EF00582E5616582602585826274F7E2
:10255B0075831E856282F0740075831EF00582E51B
:10256B00616582600B8582629060057406F0800065
:10257B00851B630222C42275831D851B82E0051B0C
:10258B0022C0D0C0E0C082C08310990C10982DD00F
:10259B0083D082D0E0D0D032C299E55BB55C05C266
:1025AB00200225C4D220855B82055B758318E0A2CF
:1025BB00E0929B758319E0F599022594E599758353
:1025CB0017855A82F07583167400A29A92E0F0A3D5
:1025DB00E5596582600385825A022594C0D0C0E01C
:1025EB00C082C083908005E030E10302268D90808D
:1025FB0005E030E2030226D8906005E030E10302EB
:10260B002622906005E030E20502266180D6D08359
:10261B00D082D0E0D0D032E5616562700990600560
:10262B007404F002260D202D1D9060027415F075B8
:10263B00831E856182E06008906000741FF0800645
:10264B00906000741BF075831E856182E0906003BF
:10265B00F0056102260D906001E075831D85648293
:10266B0020E504740080027401F0906003E0758330
:10267B001D856482F0A3E563658260038582640235
:10268B002617E55D655E700F9080057404F09080F1
:10269B000274A5F00225F99080027415F075831B66
:1026AB00855D82E06008908000741FF0800690804A
:1026BB0000741BF075831C855D82E0908003F00530
:1026CB005DB481004004000000000225F9908003F6
:1026DB00E075831A856082F0A3E55F6582600385F0
:1026EB008260022603D295C295C0E07410C39FFE90
:1026FB00600CD0E033C5F033C5F0DEF8C0E0D0E0BD
:10270B00C29020F704C2978002D297D295C295331C
:10271B00C5F033C5F0DFEBD290D295C295227A3E4D
:10272B00EAC0E0122737D0E0FADAF5227A007B20F4
:10273B00DAFEDBFC227A007B0ADAFEDBFC227A0073
:10274B007B32DAFEDBFC22000000000000080A5995
:10275B00020000000000000000000000000000006C
:10276B00000000000100040047C744E8397B396CC6
:10277B00EE00E5CDBECEBD0000000000180000004D
:10278B00008D2701014C6967687443756520202013
:10279B00202020202000020156657273696F6E2085
:1027AB00322E303020202020000101526561642040
:1027BB0000010147656E20200001062D2D3A2D2DBD
:1027CB003A2D2D2E2D2D0002014C6F636B6564206D
:1027DB0020202000020153656C662047656E202087
:1027EB000002014177616974696E6720534D505443
:1027FB0045202000020152756E6E696E6720202005
:10280B0000020149646C696E6720202020000201E0
:10281B00562D53796E632020202000020B32332E6D
:10282B0039373600020B32342066707300020B32DC
:10283B00352066707300020B333020667073000214
:10284B000B32392E39376400020B32392E39376E81
:01285B00007C
:00000001FF
